:04000000D2EF06F045
:08000800046ED8CF05F0E0CF33
:1000100006F00001E9CF0CF0EACF07F0E1CF08F0DD
:10002000E2CF09F0D9CF0AF0DACF0BF0F3CF12F01C
:10003000F4CF13F0FACF14F0F5CF15F0F6CF16F099
:10004000F7CF17F000C00EF001C00FF002C010F0A3
:1000500003C011F0F2AA30EF00F0F2B4B2EF03F0F7
:100060009DA036EF00F09EB07DEF00F0F2A63CEFD1
:1000700000F0F2B087EF03F00EC000F00FC001F007
:1000800010C002F011C003F00CC0E9FF07C0EAFF86
:10009000078E08C0E1FF09C0E2FF0AC0D9FF0BC00C
:1000A000DAFF12C0F3FF13C0F4FF14C0FAFF15C04B
:1000B000F5FF16C0F6FF17C0F7FF045006C0E0FFBB
:1000C00005C0D8FF1000F76AD60FF66E000EF722B3
:1000D0000900F5501200280C010650726F62797405
:1000E00065202020000054696D657200543D256430
:1000F0003A25303275732020000004009E903CEFBA
:1001000000F0EA6A5E0EE96EEF5011E0020E016E39
:10011000BF0E006E0400002EFDD7012EF9D7960EFB
:10012000006E002EFED700D00400EF2EEFD7120095
:10013000016A026A006A036A5A5002E1595018E0E3
:10014000100E5B6ED89057365836003603365A502C
:10015000035C02E15950005C07E35950005ED8A0EF
:1001600003065A50035ED880013602365B2EEAD76A
:100170001200996A050EC26E010E5E6EC2DFC28267
:10018000C2B2FED7C4CF03F0C350536E03C054F0C5
:1001900054C058F053C057F05A6A220E596EC8DF47
:1001A00001C027F012005F500F0B006EF00E81149B
:1001B0000010816E81880400060E006E002EFED7AE
:1001C00081981200010E5E6E9CDF5CA0819A5CB08B
:1001D000818A0400060E006E002EFED781985D38DD
:1001E0005E6E0F0E5E165EC05FF0DDDF5D500F0BC2
:1001F0005E6E5F6ED8DF818A12005C6AC00E5D6E33
:10020000E1DF12005C6A5BC05DF0DCDF12005A5077
:100210000A0A03E0020A05E009D0020E5B6EF2DF73
:100220000AD05C6A100E5D6ECDDF05D0010E5C6EEB
:100230005AC05DF0C7DF5AC001F012005A50016A7F
:10024000595C03E259C000F00CD0006A080E5B6EE6
:10025000593600365A50005CD8B0006E01365B2E1D
:10026000F7D71200200E54A8300E556E53C000F080
:1002700053AE08D0001E002A00C053F02D0E556E5C
:10028000548E5480015053C059F0640E5A6ED6DF1C
:1002900000C053F0300E0124566E53C059F00A0EC0
:1002A0005A6ECCDF300E0024586E300E0124576E8B
:1002B00055C000F0300E565C04E0548254BE5484A5
:1002C00012D055C056F0200E556E300E575C04E02B
:1002D000548054BE548207D0D8A4548004E156C040
:1002E00057F0200E566E54B405D054B206D054B018
:1002F00007D009D055C05AF08ADF56C05AF087DFC0
:1003000057C05AF084DF58C05AF081DF1200015004
:1003100057C059F0640E5A6E91DF00C057F001507B
:10032000300E07E158A20CD058B60AD058B8200EAB
:1003300003D0589658985880012601C05AF067DFBC
:1003400057C059F00A0E5A6E79DF00C057F00150BD
:10035000300E06E158B608D058A006D058B8200E86
:10036000012601C05AF053DF300E572657C05AF00D
:100370004EDF12000900F6CF58F0F7CF59F0F5CF55
:100380005AF045DF58C0F6FF59C0F7FF572EF2D795
:10039000120033DF540E5A6E3ADF3D0E5A6E37DFCD
:1003A00027C053F0180E546E5DDF3A0E5A6E2FDFE1
:1003B0001EC057F0010E586EAADFF50EF66E000E45
:1003C000F76E030E576ED6DF120059505B02F3CF63
:1003D00001F0F4CF00F05C02F35000265A505B02AB
:1003E000F3500020026E12000900F6CF58F0F7CF4C
:1003F00059F0F5509EA8FED7AD6E58C0F6FF59C013
:10040000F7FF572EF1D71200015057C059F0640E74
:100410005A6E14DF00C057F00150300E07E158A2A9
:100420000DD058B60BD058B8200E03D05896589817
:100430005880012601509EA8FED7AD6E57C059F0D6
:100440000A0E5A6EFBDE00C057F00150300E06E176
:1004500058B609D058A007D058B8200E0126015030
:100460009EA8FED7AD6E300E572657509EA8FED7D9
:10047000AD6E1200EACF5FF0E9CF5EF058AE08D063
:100480005E8E5EA85E2A571E581E572AD8B4582A78
:100490005838F0095A6E5A26E20F5B6E320F5D6EC5
:1004A00058500F0B5B265B265D26E90F5C6E5C26C1
:1004B0005C2657380F0B5C265D265C365D365D1E6C
:1004C0005D3657500F0B5D265A36070E596E0A0ED1
:1004D0005C065D26FDE35B065C26FDE35A065B26B3
:1004E000FDE359065A26FDE3EA6A590EE96E070E46
:1004F0005E145E9CED525E1407E15EB8EE525EB88B
:1005000003D0200E006E20D0E926000EEA22E9502A
:100510005D0803E1EA5201E15E8CEF50006E08E1F4
:100520005EBC06D05EB814D05EB602D0200E0BD0F2
:100530005EAE06D02D0E006EED505E9C5E9E04D029
:100540005E865E98300E002600509EA8FED7AD6EE7
:10055000EE505EACDCD712005C6A800E5D6E32DE5F
:1005600012000900F5520CE0F6CF57F0F7CF58F023
:10057000F5CF5AF04CDE57C0F6FF58C0F7FFF1D761
:100580001200996A050EC26E010E5E6EBADDC2825D
:10059000C2B2FED7C4CF03F0C3501C6E03C01DF01F
:1005A00024C05AF023C059F05C6A090E5B6E0DDF5F
:1005B0001C500124236E1D500220246E24C058F0CC
:1005C00023C057F05A6A0A0E596EB2DD02C024F0F9
:1005D00001C023F024C058F023C057F05A6A0A0E15
:1005E000596EA6DD01C056F0B80EF66E070EF76E16
:1005F000070E576EF9DE56C057F01B0E586E04DF1B
:10060000556A55500F080DE3036A5550330FE96ED4
:10061000000E0320EA6EEF50565C01E202D0552A2C
:10062000F0D73C0ED88055541C6E1D6AC20EF66E73
:10063000070EF76E030E576ED7DE55C057F01B0E30
:10064000586EE2DEC70EF66E070EF76E050E576E99
:10065000CBDE100EE96E1DC058F01CC057F00ADF4B
:10066000200E9EA8FED7AD6E1DC058F01CC057F0DE
:100670005A6A0A0E596E5CDD01C053F0586A53C0C5
:1006800057F058C05AF053C059F05C6A0A0E5B6EBE
:100690009CDE01501C5C006E02501D5800C054F0DE
:1006A0005BDFD20EF66E070EF76E5BDF53C057F0BE
:1006B0001B0E586E2CDE2E0E5A6EA9DD54C057F05C
:1006C0001B0E586E24DEDD0EF66E070EF76E050E5D
:1006D000576E50DEE40EF66E070EF76E060E576E7E
:1006E00083DE53C057F01B0E586E8EDE2E0E9EA872
:1006F000FED7AD6E54C057F01B0E586E85DEEF0E60
:10070000F66E070EF76E050E576E6EDE120081BC98
:100710001FD02FDD640E5E6EF4DC81BC13D01B5243
:1007200007E01E2A1E503B0802E23B0E1E6E05D05B
:100730001E5202E01E0601D01E6A2BDEC80E5E6E3F
:10074000E0DCEBD71B5202E01B6A02D0010E1B6EED
:1007500081BE05D016DF1F6A020E2724206EF2909C
:100760003CEF00F0E10ED76E800ED66E322A275293
:1007700005E11E5203E1010E1F6E1BD01E061E5026
:100780003B0801E21E6A1E5214E1275212E03C0EA1
:100790001E6E2550261004E02550D8B426062506E6
:1007A000205202E0200602D0010E1F6E275201E007
:1007B0002706F2943CEF00F00D20626174743D2531
:1007C00075000D693D25752042415420256C64203B
:1007D00000004241543D000025752E25755620200D
:1007E00020200000200D4241543D25752E257556D0
:1007F00020202020000042415454204C4F5720001C
:100800000D2062616466696C6572203D256C75001F
:100810000D4F483347444F20200031322D737979F2
:10082000732D3136000054696D65722039363030D1
:10083000206261756420200054696D65722020007B
:1008400054696D6572202020000025643A253032FD
:100850007573202020000D4261747465727964699B
:10086000706C617954696D65723D256C64000D2072
:1008700054696D653D25640054696D65206F75741C
:100880002000C00E936E819A8198196AF2BE198E6B
:10089000F29E0F0E5E6E35DC19BEF28E010E466EB4
:1008A0004650030814E3196AF2BE198EF29E030E35
:1008B0005F6E79DC19BEF28E196AF2BE198EF29E55
:1008C000050E5E6E1EDC19BEF28E462AE9D7196A45
:1008D000F2BE198EF29E020E5F6E65DC19BEF28EBC
:1008E000466A4650030810E3036A465063EC00F082
:1008F000476E196AF2BE198EF29E5C6A5D6E62DC0A
:1009000019BEF28E462AEDD7196AF2BE198EF29EF2
:100910005C6A0D0E5D6E56DC19BEF28EC0EF04F0FF
:10092000B990C19CC19E030EB86E000B01099A6E6E
:10093000C050800B0709C06EC294C296C298C29A7A
:10094000C08EC198C280996A050EC26EC66AF19EB9
:10095000870ED56EA50ECD6EF00EBA16BD16DF0E43
:10096000926EC00E936E300E946E8168806AC00ED7
:10097000826E94968B86F28AF2869D80F21281D7DF
:10098000266A0A0E256E17EF07F0EACF4FF0E9CF7F
:100990004EF04838F0094A6E4A26E20F4B6E320F8D
:1009A0004D6E48500F0B4B264B264D26E90F4C6ED3
:1009B0004C264C2647380F0B4C264D264C364D36D0
:1009C0004D1E4D3647500F0B4D264A36070E496EC9
:1009D0000A0E4C064D26FDE34B064C26FDE34A0667
:1009E0004B26FDE349064A26FDE3EA6A490EE96E15
:1009F000070E4E144E9CE926000EEA22E9504D08DF
:100A000003E1EA5201E14E8CEF50006E08E14EBC6A
:100A100006D04EB80CD04EB602D0200E03D04E8673
:100A20004E98300E002600509EA8FED7AD6EEE50B8
:100A30004EACE4D762EF05F00A0E466E996A010EDD
:100A4000C26E196AF2BE198EF29E010E5E6E81ECC4
:100A500000F019BEF28E246A236A46504606000A48
:100A60000AE0C282C2B2FED7C4CF03F0C35023262D
:100A700003502422F2D7196AF2BE198EF29E24C0C6
:100A800058F023C057F05A6A0A0E596E98EC00F0DD
:100A900019BEF28E02C024F001C023F0000EF66EE3
:100AA000080EF76E196AF2BE198EF29E0C0E576E82
:100AB0009BDC19BEF28E100EE96E24C048F023C0F4
:100AC00047F063D719EF07F00900F5520DE0F6CFB4
:100AD00046F0F7CF47F0F5509EA8FED7AD6E46C062
:100AE000F6FF47C0F7FFF0D71200100EF66E080EA3
:100AF000F76EEADF200E9EA8FED7AD6E1A0EF66ED8
:100B0000080EF76EE1DF0D0E9EA8FED7AD6E260E25
:100B1000F66E080EF76ED8DF22EF07F0196AF2BE04
:100B2000198EF29E5C6A010E5D6EE2EC00F019BE59
:100B3000F28E9CEF05F0F2D7196AF2BE198EF29E82
:100B40000BDD19BEF28EDA0EF66E000EF76E196A24
:100B5000F2BE198EF29E05DD19BEF28E196AF2BE42
:100B6000198EF29EFDEC00F019BEF28EE60EF66EC6
:100B7000000EF76E196AF2BE198EF29EF2DC19BEF3
:100B8000F28E23EF07F0996A010EC26E196AF2BE67
:100B9000198EF29E010E5E6E81EC00F019BEF28E8F
:100BA000C282C2B2FED7C4CF03F0C350466E03C0A8
:100BB00047F0196AF2BE198EF29E47C058F046C03F
:100BC00057F05A6A0A0E596E98EC00F019BEF28E70
:100BD00002C01DF001C01CF01D522FE11C50310855
:100BE0002CE322522AE1196AF2BE198EF29EFDEC24
:100BF00000F019BEF28EF60EF66E070EF76E196A49
:100C0000F2BE198EF29EADDC19BEF28E196AF2BEEA
:100C1000198EF29EB6DC19BEF28E080E466E196A67
:100C2000F2BE198EF29EFA0E5E6E81EC00F019BED5
:100C3000F28E462EF4D7010E226E87EF07F0200EBB
:100C400047A8300E486E46C000F046AE08D0001EE1
:100C5000002A00C046F02D0E486E478E4780015096
:100C6000196AF2BE198EF29E46C059F0640E5A6E91
:100C70001EEC01F019BEF28E00C046F0300E0124C9
:100C8000496E196AF2BE198EF29E46C059F00A0EDC
:100C90005A6E1EEC01F019BEF28E300E00244B6E1F
:100CA000300E01244A6E48C000F0300E495C04E06A
:100CB000478247BE478412D048C049F0200E486E94
:100CC000300E4A5C04E0478047BE478207D0D8A474
:100CD000478004E149C04AF0200E496E47B405D070
:100CE00047B207D047B009D00CD048509EA8FED7D5
:100CF000AD6E49509EA8FED7AD6E4A509EA8FED755
:100D0000AD6E4B509EA8FED7AD6EC7EF07F0090E33
:100D10004B5E0BE3EA6A4B0EE96ED890EF32EF5070
:100D200004E001D00400EF2EFDD71200496A486AA2
:100D3000495236E14850020833E3476A466A475051
:100D400001081CE303E14650F30818E394948B84F4
:100D50000400020E4A6EF70E4B6ED9DF4A2EFBD707
:100D600094948B940400020E4A6EF70E4B6ECFDF04
:100D70004A2EFBD7462AD8B4472AE1D7040E4A6E3A
:100D8000196AF2BE198EF29EFA0E5E6E81EC00F0C8
:100D900019BEF28E4A2EF4D7482AD8B4492AC8D7A9
:100DA000D4EF07F0F86AD09E078E720ED36E9B6A5E
:100DB000D3501A6A010E1B6E1D6A1C6A010E1E6E4C
:100DC0001F6A050E206E216AAA960C0EAF6EA20E47
:100DD000AC6E900EAB6E226A246A236A316A306A66
:100DE000326AB990C19CC19E000EB86E286A296A09
:100DF000270E336E280E346E290E356E2A0E366E8F
:100E00002B0E376E2C0E386E396E2D0E3A6E3B6EF1
:100E10003C6E2F0E3D6E300E3E6E310E3F6E406EBC
:100E2000416E320E426E330E436E816879D58286F2
:100E300003D6196AF2BE198EF29EC1EC02F019BEF9
:100E4000F28E53D678D6196AF2BE198EF29EB9EC9C
:100E500000F019BEF28E196AF2BE198EF29EACEC49
:100E600002F019BEF28E380EF66E080EF76E196A91
:100E7000F2BE198EF29EB1EC02F019BEF28E400E57
:100E8000F66E080EF76E20DE196AF2BE198EF29E1B
:100E9000FDEC00F019BEF28E196AF2BE198EF29EB8
:100EA00027C053F0180E546E32EC01F019BEF28ECA
:100EB000196AF2BE198EF29E3A0E5A6E07EC01F0D4
:100EC00019BEF28E196AF2BE198EF29E1EC057F03C
:100ED000010E586E87EC01F019BEF28E510EF66EBF
:100EE000080EF76E196AF2BE198EF29E040E576E46
:100EF000BAEC01F019BEF28E325226E0196AF2BE47
:100F0000198EF29EC9EC01F019BEF28E3CD6560E37
:100F1000F66E080EF76E196AF2BE198EF29E140E66
:100F2000576EF4EC01F019BEF28E100EE96E196ADC
:100F3000F2BE198EF29E26C058F025C057F03AEC4A
:100F400002F019BEF28E326A255026100BE1266A95
:100F50000A0E256E196AF2BE198EF29EC1EC02F0DD
:100F600019BEF28E1F5223E06E0EF66E080EF76E5B
:100F7000196AF2BE198EF29E070E576EF4EC01F05C
:100F800019BEF28E1FC046F0180E476E58D6780E66
:100F9000F66E080EF76E196AF2BE198EF29EB1EC6B
:100FA00002F019BEF28EC2D61F6A94968B96A4D711
:020FB00003003C
:0200000400F00A
:09000000504F5945204B4E393197
:020000040030CA
:0E00000000C80E2F3C1D81000FC00FE00F4006
:020000040020DA
:080000000000060001000200EF
:00000001FF
